:030000000219FDE5
:03000B000200AA46
:03002B000201636C
:03005B000202FDA1
:030073000202EA9C
:1000800002030406080C10182030406080040608A3
:100090000C10182030406080A0C00003070F1F0D17
:1000A0000D04050D050305030302C2AFC0D0C0E077
:1000B000206214E5256009E473E525F4F58AD2622F
:1000C000D0E0D0D0D2AF3285268AC262E526F46075
:1000D0003630682C20720DD0E0D0D0C283C294C2DA
:1000E00095D2AF32C283C294C295206F132065109F
:1000F000740CD5E0FDE57BB4800442902100428081
:10010000D0E0D0D0D2AF32758A00C28DD262210049
:1001100001B9306805206502D28301B93068052035
:100120006502D29401B9306805206502D29501B903
:10013000C28030680A2065077408D5E0FDD28301CB
:10014000B9C28230680A2065077408D5E0FDD294F0
:1001500001B9C29730680A2065077408D5E0FDD25E
:100160009501B9C2AFC2AD53E6EFC0D0C0E0D2D363
:10017000D2AFC2CEE52A600720744F152A21CA7873
:1001800000790020742EE580307E01F430E502789D
:10019000FF53DACF207E0343DA20307E0343DA10A8
:1001A000C2D8C271E580307E01F430E50279FFC328
:1001B000E89970CB306103752A18207403752A18EA
:1001C000885CD270E86003755F0020740DE52B60D9
:1001D00004152B21DA43DA01C2D82070024149A864
:1001E0005C206102C2702074367982B70431C3E8A2
:1001F00094F0400374F0F8E8C4540F28F87984B7F9
:100200000302411FC313C3138721200802C3132015
:100210000A06C3C898F8411F28F8500374FFF888ED
:1002200022E52D54066022206B1FE536C333C3330D
:10023000F8E564C313C313F9C3952240028922E889
:100240002522F52250037522FF7882B604598522B3
:1002500024A824C3E52495614002A861C3E89563FE
:100260004002A8638825E5667002419AC3E8AA6641
:100270009A5003E8FAE4F9EAC333FBE568F45B2932
:10028000400D2567F8E56760021567400B419A0A43
:10029000C3E5679A5002056778FF8826C26FC3E5F9
:1002A0002694F84002D26F20CF0AD0E0D0D043E6A7
:1002B00010D2AD32C2CF053A7801E52A600530741C
:1002C00002152AC3E55C94014005755F0041E075A5
:1002D0006000756900E55F2401F55F5003755FFFFD
:1002E000D0E0D0D043E610D2AD32C2AF53E67F7536
:1002F00092FA7593FFC260759104D2AF32C2AF53C8
:10030000E6EFC2ADC0D0C0E0C0F0D2D3D2AFA8FB00
:10031000A9FCC2D8307102616453DACF207E034356
:10032000DA10307E0343DA20D271E580307E01F4AA
:1003300020E502613B88278928A19153DACF207EEE
:100340000343DA20307E0343DA10C2D8C27130741E
:1003500002A17D7800E580307E01F430E502A17DC8
:10036000885CA16553DACF207E0343DA20307E0318
:1003700043DA10C271206102813D53DACF207E033F
:1003800043DA10307E0343DA20C2D8D2718857890D
:1003900058C3E89555F8E99556F97B007E087A0030
:1003A000C3E8948CE994005005755B00812F882187
:1003B00078A2E6A8216055C3E894C8E994005008E3
:1003C000E4D2E4FB7A0A810AC3E89468E994015014
:1003D00008E4D2E3FB7A0F810AC3E894D0E99402DF
:1003E0005008E4D2E2FB7A1E810AC3E894A0E994A3
:1003F000055008E4D2E1FB7A3C810AC3E89498E90D
:1004000094085008E4D2E0FB7A787E00C3E895595E
:10041000FCE9955AFD30E70AECF42401FCEDF434D4
:1004200000FD755B00C3EC9AED9E5003755B01887F
:1004300059895A8557558558567802A165C3E8955C
:1004400027F8E99528F9307C02A149307B02A149BF
:10045000307A02A1422075028160E9FDE8FC817FCB
:10046000E9C313F9E813F8307902A142E9C313F99B
:0F047000E813F8307802A142E9C313FDE813FC4A
:10047F0020612CC3EC941CED940240028196ED7028
:10048F001EC3EC94C850180529E52970021529C31D
:10049F00E529940A5002A17D755C00D270A17DE51B
:1004AF0029600215297888E6F97400207F0878966C
:1004BF00B90302789EE624FAFEE43400FFC3EC9EF3
:1004CF00FCED9FFD9208B90310A208500720760992
:1004DF00D27681E8307602C276A2085016B9030DA3
:1004EF00ECF42401FCEDF43400FD020502780079F0
:1004FF0000A149B90315EC33FCED33FDC3EC940AAD
:10050F00FCED9400FD50047C007D00C3EC94FFEDE6
:10051F009400400678FF7900A149EC8572F0A4C5DC
:10052F00F0A2F733F87900400302056578FF7900F0
:10053F00020565E9C313F9E813F8307C0EE9600290
:10054F0078FFC3E81338F8E43400F9C3E894FFE9FF
:10055F009400400278FF885CD270206102A17D7404
:10056F001FF4552F4BF52FC274EB7002D274752AFE
:10057F0018307403752A0A306102A1912074035355
:10058F00DAFE207403752B06D0F0D0E0D0D0D2ADB8
:10059F0043E6103279010205C179030205C1790AD8
:1005AF000205C1791E0205C179640205C179C8022D
:1005BF0005C17817E4D5E0FDD8FAD9F6227A147B75
:1005CF00780205E87A107B8C0205E87A0D7BB4027D
:1005DF0005E87A0B7BC80205E8E573D5E0012279BF
:1005EF0002E4C282D5E0FDD294D5E0FDC294D5E0FD
:1005FF00FDD282D5E0FDE920E002D28330E002D2C5
:10060F0095E573D5E0FDE920E002C28330E002C238
:10061F00957496D5E0FDD9C9EAF8D5E0FDD8FBDB96
:10062F00B8C28222C37C007D0075F00005F0EA336A
:10063F00FAEB33FB50F6EB13FBEA13FAC3E9FFE8CF
:10064F00FEE89AF8E99BF95004EFF9EEF8B3EC33B2
:10065F00FCED33FDD5F0DFEDF9ECF822E889F08AF7
:10066F0020D2D4F8A9F07B0030F70B7BFFF42401E4
:10067F00F8E9F43400F9E88520F0A4ADF0F8E98545
:10068F0020F0A4AFF0FEED2EF974003FFA7C04C306
:10069F00EA13FAE913F9E813F8DCF48BF030F70AF0
:1006AF00E8F42401F8E9F43400F9E889F0C2D4F849
:1006BF00A9F0227882B6040302071DC3E55C9401FA
:1006CF0040030206E7852224E4F544F545F546F597
:1006DF0047F548C26E02071D7882E6FCD26EE5220E
:1006EF00F523783879C7AA40AB41C3EB13FBEA1364
:1006FF00FAEC146013C3EB13FBEA13FAEC14146057
:10070F0007C3EB13FBEA13FAD1338844894522C39D
:10071F00E5449523F8E5459400F9500CC3E894801F
:10072F00E994FF401602074EC3E8947FE994005006
:10073F000302074E787F790002074E788079FF8891
:10074F0049894A22E5492546F8E54A3547F9854A58
:10075F0020E4300701F43548FA30E709C3EA94F092
:10076F00401502078CC3EA940F500302078C78FFE1
:10077F0079FF7A0F02078C780079007AF0C3E524AD
:10078F009561500AC374019524500B0207AAE54ADC
:10079F0020E70E0207AAE54A30E706884689478A0E
:1007AF00482278A5E6FAC3E54933F8E54A33F9D18B
:1007BF006BE930E70BC3E89480E994FF4013E1E461
:1007CF00C3E8947FE994005002E1E4787F7900E177
:1007DF00E4788079FFE820E715C3E52398F840090E
:1007EF00C3E89401400302080B780102080BE8F4F8
:1007FF0024012523F8400302080B78FF884B227849
:10080F00A6E6FAA847A94812066BE930E70CC3E839
:10081F009401E994FF4016020840C3E894FFE9945D
:10082F0000500302084078FF7900020840780179F0
:10083F00FFE920E715C3E54B98F84009C3E8940199
:10084F0040030208677801020867E8F42401254B8A
:10085F00F8400302086778FF88242278FF20692870
:0F086F0079A1E76023E541601F74FF8541F084A4
:10087E008539F0306A0375F005A4F8C5F06002788A
:10088E00FFC3E895645002A864886322C3E54094D0
:10089E0040E5419401E56350031401AB046002F599
:1008AE0063220208B32275E890227883E6FF30EDCA
:1008BE00F9A8BDA9BE0570C3E570940840527570C5
:1008CE0000E9FA79A0E76044EA7007E571601B025F
:1008DE0008ECC3E895716010E5715006600C1402C7
:1008EE0008F80460F90208F8E571F571C3946D40DB
:1008FE001B7561C0C394044013756180C39404409A
:10090E000B756140C39404400375610075BB0922E9
:10091E00E5612410500274FFF5617982B70402215B
:10092E0045C3A861E524985002A824C3E895634006
:10093E0002A86388258826E570B4070375BB1022CC
:10094E00743279A787F0A4C5F0A2F733F8C3E895FF
:10095E00614002A86188228824882588268864221E
:10096E007540007541F022C2AF75C820A8CCA9CD44
:10097E00AA3A30CF010A75C824D2AFAB3BAC3C8843
:10098E003B893CC3E89BF8E99C206908F930660274
:10099E00418621E0AD3D8A3DF9EA9DFA600678FF79
:1009AE0079FF21C5AE3EAF3F8B3E8C3FA83BA93CA5
:1009BE00C3E89EF8E99FF9C3E54113FBE54013FA3E
:1009CE00E82AF540E93BF54150067540FF7541FFB9
:1009DE00412DAA40AB41AC40AD417E047F02C3EB3A
:1009EE009404400D1E1FC3EB94084005206A021E9E
:1009FE001FC3ED13FDEC13FCDEF7C3EA9CFAEB9D6F
:100A0E00FBEF6009C3E913F9E813F8DFF7EA28FAF8
:100A1E00EB39FB8A408B4150067BFF8B408B41C3E9
:100A2E00EB94025002D2663069047F0341587892EB
:100A3E00E6FFC3E537948240110FC3E53794A0401B
:100A4E00010FC3EF940640027F057E02E541C454B8
:100A5E000FF9E541C454F0F8E540C4540F28F8C32B
:100A6E00E89EFAE99400FB4009C3EA9402EB940075
:100A7E0050047A02E4FB41D2AA40AB41EBC4FEEA39
:100A8E00C4540F4EFCC3EA9CFAEB9400FBC3E8136C
:100A9E00C313F8EA28FAEB3400FB8A408B41C3EB10
:100AAE0094024002C2667802EBC4FE7B00EAC45494
:100ABE000F4EFAC3EA98FA4005C3940250027A0226
:100ACE007892E6FF30600241D2855192855293D2E0
:100ADE006043E680C3E49AF8E49BF9306602615EF7
:100AEE00E8FAE9FBD3E913FDE813FC88518952C3F8
:100AFE00EF94036038EF20E00DE82CF8E93DF9ECB7
:100B0E00FAEDFB020B27E828F8E939F9C3E82402CD
:100B1E00F8E93400F97AFE7BFFC3EF9403400E8AA6
:100B2E00538B54884D894E8C4F8D506192885389CA
:100B3E00548A4D8B4E8C4F8D503069127553F07513
:100B4E0054FF754FF07550FF7551F07552FF61925D
:100B5E00E8FAD3E813FC8851C3EF94036020EF202A
:100B6E00E007E82CF8ECFA617EE8282402F87AFE19
:100B7E00C3EF940340088A53884D8C4F619288537B
:100B8E008A4D8C4FE568C3335002646BF568306054
:100B9E0002619C753402D26043E680E52D540660F6
:100BAE0034A840A941C3E913F9E813F8C3E913F9CE
:100BBE00E813F8306904E92440F9C2AF53E67F75B3
:100BCE009100C3E498F594E499F595759104D2607B
:100BDE0043E680D2AF22D264754300752000306C9C
:100BEE0003752040020C03D264754300752040301B
:100BFE006C0375200078017901206620E52D5406DE
:100C0E006002C2647914E541C313700104F8C39401
:100C1E001440027814306904781B791B206010E5AB
:100C2E0043600C306903D53404D26D81AE71A405D6
:100C3E0043E59BF45440B52002819830690908C3FE
:100C4E00E899400118812A20640A08C3E8994002F5
:100C5E008103812AC264C2AF53E67F75910030666C
:0F0C6E00127594007595F8759104D26043E68075
:100C7D00D2AF8103E5417EFFC3334005C33340014D
:100C8D00FEC3E49E759400F5958175C3E53394011B
:100C9D00500281033064028103D80281AC812AC2E3
:100CAD006DC2AF53E67F759100855394855495754C
:100CBD009104854D92854E93D26043E680D2AFE587
:100CCD002D54066008206A020533020CEA306D0DC2
:100CDD00206C0A206407158115810215AB2278005E
:100CED003064027801E53775F007A4F9E5F028F5D1
:100CFD00F0E9A2F013A2F113A2F213F537C3947821
:100D0D005003753778C3E53795384008D265C283EF
:100D1D00C294C295306002A121854F92855093D225
:100D2D006043E68022207D16C2AF754202C282D298
:100D3D0080306202D295D2AF759F43020F22C2AFAF
:100D4D00754202C282D297306202D283D2AF759FB2
:100D5D0043020F22307243207D20C2AF75420390B3
:100D6D000141757B04C295C297306204D294A17F74
:100D7D00D282D2AF759F53020F22C2AF754203903C
:100D8D000141757B04C283C280306204D294A19F5D
:100D9D00D282D2AF759F33020F22207D17C2AF755D
:100DAD00420390011CC295306202D294D2AF759F5E
:100DBD0053020F22C2AF75420390011CC2833062F1
:100DCD0002D294D2AF759F33020F22207D16C2AF8F
:100DDD00754204C280D297306202D294D2AF759F11
:100DED0033020F22C2AF754204C297D28030620225
:100DFD00D294D2AF759F53020F22307243207D20C3
:100E0D00C2AF754205900130757B01C294C282302C
:100E1D006204D283C125D280D2AF759F43020F22C7
:100E2D00C2AF754205900152757B80C294C282306B
:100E3D006204D295C145D297D2AF759F43020F225E
:100E4D00207D17C2AF754205900112C29430620227
:100E5D00D283D2AF759F43020F22C2AF7542059068
:100E6D000126C2943062EBD295D2AF759F43020F2B
:100E7D0022207D16C2AF754206C297D28230620221
:100E8D00D283D2AF759F53020F22C2AF754206C2F5
:100E9D0080D282306202D295D2AF759F33020F227B
:100EAD00307244207D20C2AF754201900152757B96
:100EBD0080C283C280306204D295C1CBD297D2AFAB
:100ECD00759F33020F22C2AF754201900130757BC1
:100EDD0001C295C297306205D283020EECD280D248
:100EED00AF759F53020F22207D17C2AF754201903F
:100EFD000126C283306202D295D2AF759F33020FA5
:100F0D0022C2AF754201900112C295306202D283A6
:100F1D00D2AF759F53C26522900110757B00C283BD
:100F2D00C294C295C280C282C297C2622278807674
:100F3D00090876090876040876FF0876030876FF17
:100F4D00087609087603087601087601788C760113
:100F5D000876FF0876FF0876FF0876FF0876FF080B
:100F6D0076030876FF0876FF0876FF087625087663
:100F7D00D00876280876500876040876FF087602A1
:100F8D0008760008767A0876FF087601087601085B
:100F9D007600087603087600227887E6FFC272BFD6
:100FAD000302D2727888E6C394036008C27DE630EE
:100FBD00E102D27DC27E7889E630E102D27EC3EFB6
:100FCD0094026008758E01D273020FDE758E00C219
:100FDD0073227880E6149000809378A5F67881E6E8
:100FED00149000809378A6F67886E61490008D9381
:100FFD0078A7F67886E6F539C39402500375390261
:10100D00789CE67538FFB402037538A0B4030375F8
:10101D00388278A3E61490009A93F566120F252274
:10102D00D281789DE66002C281227896E6FA7897A1
:10103D00E6FB7888E6B40305C3EB940EFB307F0422
:10104D007A007BFFC3EB9AFCC3948250027C8275BD
:10105D0072000572EC8572F0A4C3E5F0947D40F248
:0F106D0022D27F11371205B21205B27A007B0032
:10107C007C101205A8E55C2AFA74003BFBDCF37CBF
:10108C0004C3EB13FBEA13FADCF7FEC27F11372221
:10109C00757C00757D00E5EF20E6037520000520CA
:1010AC00903FFFE520146006901DFF146000930430
:1010BC00600375EF1653D9BF7581C043FF801205CD
:1010CC00A375EF0643B203E5B3240220E70DF52127
:1010DC00E5E320E0068521B343E301120F2575807B
:1010EC00F075A40F75F13F75D4DF75904F75A5B0F1
:1010FC0075F2F575D50075A60175E241120F25E460
:10110C00F8F6D8FD756801120F3A1215FC7898861E
:10111C0073753001C2AF1205BC1205CC1205B212A8
:10112C0005D31205B21205DA1205B2C2AF757C00F6
:10113C00757D0078FA79FA308507D9FBD8F7021C4F
:10114C0000120FA6120FDF112D113778988673122B
:10115C000F2575881075890275C82475910475D88A
:10116C004075A82275B80275E690759B80759D0038
:10117C0075D10E75BC5875BB0975BA1175E880121E
:10118C0005A3D2AF1208B075360053DACF207E0318
:10119C0043DA20307E0343DA1043DA01C2D8C2713D
:1011AC001205BCD2617B037A0CE55B70077A0CDB11
:1011BC00030211371205B2207003021137C270E519
:1011CC005CC3940240E1E52F541F855E5DF55EB56E
:1011DC005DD5DAD5C26153DACF207E0343DA2030F5
:1011EC007E0343DA10C2D8C27178A2E67008D274BA
:1011FC00E52F54E0F52FC2757529001205B7307430
:10120C0009C3E529940A4002D2751205A878023068
:10121C0074027800C3E55C9840F0C2AF1205CC12A2
:10122C0005CC1205CCD2AF1205BC754C007888E603
:10123C00B40302612C1205A8788CE6C39401500308
:10124C0002132CE530C39401500302132C757CA5BA
:10125C00757DF1207435C3E55C94FF500302132CAB
:10126C00C2AF1205E1D2AF1205B7C3E55C940150D1
:10127C00EFC2AF1205CC1205AD1205CCD2AF1205E0
:10128C00B7C3E55C94FF40E90217B47F02D27F112B
:10129C00371205B7C2AFC27F1137AE5CC3E55C94A1
:1012AC007FD2AF5002613C1205A3C2AF1205E1D24E
:1012BC00AFDFDA116EC3EE7897F61205BC12173752
:1012CC007F0AD27F11371205B7C2AFC27F1137AE7A
:1012DC005CC3E55C947FD2AF50E61205A3C2AF129B
:1012EC0005CC1205AD1205CCD2AFDFD6116EEE24B3
:1012FC00037896F6F87997E7C394824003985006E2
:10130C00E824827897F61205BC12164A1217661258
:10131C0005B71137C3E55C94FF500241590217B46D
:10132C00757C00757D00C3E55C954C4003855C4C79
:10133C001205B778017988E7B403027805C3E55C38
:10134C009840024139C2AF1205E11205E11205E1E4
:10135C00D2AF1205BC753000E4F531F5320531E53C
:10136C0031F4703F0532789AE678191460127832AD
:10137C0014600D787D14600878FA146003753200DF
:10138C00C3E53298401D120F251205A31532753195
:10139C000078998673C2AF1205E1D2AF7898867344
:1013AC001205B71205ADE52A7005307402213778A5
:1013BC00012074027806C3E55C9840A17888E6C3E6
:1013CC00940360031205B7E52A7003021137C2AF0C
:1013DC00120F25E4F522F523F524F525F526F567FE
:1013EC00D2AF7885E6C333F565E4F544F545F546AB
:1013FC00F547F548F570F52CF52DF5377570087532
:10140C00BB101205A31208B430EDFDA8BDA9BEE9AE
:10141C007001F888711208B875700875BB10120F3E
:10142C00A6C2AF7561FF12094E85226185226285C5
:10143C002263D2AF75220175240175250175260131
:10144C00856069756A017888E6B40307C27D3076D9
:10145C0002D27DD268D269753300120E7E120EADA7
:0F146C0012096E12097512096E12097512096EB6
:10147B00120BF51206C2120CEB120D321209751279
:10148B000BE4306E0312071E20660312086A3066E7
:10149B000312089A120CEB120D61120975120BF55F
:1014AB00306E03120753120CEB120DD81209751282
:1014BB000BE4306E031207B1120CEB120E0712097C
:1014CB0075120BF5306E0312080E120CEB120E7E1A
:1014DB001209751208B4120BE4120CEB120EAD12BA
:1014EB0008B812097530693285646185646285605C
:1014FB0069756A0179187A0CC3E53399400FC26993
:10150B00D26A8A35856461856463021525C3E55CFF
:10151B009401400302147B0215B3306A25206C2220
:10152B00E535147006C26AD26B817BF535C3E55C79
:10153B009401400302147B7888E6C3940360030292
:10154B0015B375360078FA79A4E760027803C3E522
:10155B005F985054307404E52A604D7888E6B403E4
:10156B0017207D05207607A183307602A183206C9E
:10157B0007D26C85646181BA78F0306C0585646143
:10158B007820C3E541985002817B306C1BC26CC242
:10159B007D307602D27DD26A753512856461817B8E
:1015AB000536E55C6002A1B6753600C2AF120F2599
:1015BB007887E6FE7602120FA67887EEF6E4F52220
:1015CB00F523F524F525F526F565752C00752D000D
:1015DB00D2AF1205B7120F2578A4E66006D283D2DC
:1015EB0094D295307409C3E53694044002213761D7
:1015FB0064901A0D782012168CE520B4550CA312AA
:10160B00168CE520B4AA0302162A757CA5757DF10C
:10161B00120F3A12164A757C00757D00021649901E
:10162B001A0378807B0A12168CA308DBF9901A0F29
:10163B00788C7B1912168CA308DBF9901A2822C21E
:10164B00AF1216CF1216AC901A00740E121691A38D
:10165B007409121691A37415121691901A037880BF
:10166B007B0A121690A308DBF9901A0F788C7B1962
:10167B00121690A308DBF91216E21216C0901A2864
:10168B0022E493F622E6438F01538FFDFFC3E583DC
:10169B00941C400122EF857CB7857DB7F0538FFEFC
:1016AB0022438F02438F01857CB7857DB7901A0D3E
:1016BB00F0538FFC22901A0D7455D191901A0E7421
:1016CB00AAD191227A3079D07820901A40D18CE52A
:1016DB0020F709A3DAF7227A3079D0901A40E7D1B4
:1016EB009109A3DAF922AB74A875BB01027980BB0F
:1016FB0002027981BB03027982BB04027984BB05A8
:10170B00027986BB06027992BB07027987BB080276
:10171B0079A3BB0902799CBB0A027988BB0B0279BE
:10172B0089E8F7227C051205BCDCFB22C2AF12054F
:10173B00CC1205D31205DA1205E11205AD1205CC58
:10174B001205D31205DA1205E11205AD1205CC1202
:10175B0005D31205DA1205E1D2AF22C2AF1205E1B1
:10176B001205DA1205D31205CC1205AD1205E112E2
:10177B0005DA1205D31205CC1205AD1205E11205DF
:10178B00DA1205D31205CCD2AF22AE74AF75C2AF4D
:10179B001205CC1205CC1205CC1205ADDEF21205EA
:1017AB00E11205ADDFF8D2AF22F137F12FF12F7532
:1017BB007401757501757600F1957C05AD5C1205AC
:1017CB00BCC3ED955C70F5C3E55C9401400AC3E5C1
:1017DB005C94FF40320217F0D1F1D14AF137C2AF1E
:1017EB0075EF16F12FDCD50576C3E5769403500221
:1017FB0080C6F12F0575E5741490009F93F808C30C
:10180B00E57598500280AE12172F12172F0574C36F
:10181B00E574940C5002809A120F3A12164AC2AF1A
:06182B0075EF1612172FE5
:0319FD0002109C39
:101A00000E0915090904FF03FF0903010155AA0185
:101A1000FFFFFFFFFF03FFFFFF25D0285004FF0259
:091A2000007AFF0101000300FF40
:101A400023416C69676E424C33355023202020209F
:101A500023424C48454C4923463333302320202031
:101A60002020202020202020202020202020202076
:101C0000C2AFC2D353D9BF7581C043B20343FF8073
:101C1000752438752503B1DC7529A5752AF175E29F
:101C20004043F12053A4DF75D4FFD2857DFA7803B9
:101C300079E67C10752200752300901DE97B0675FE
:101C400024987525013085028145208508D8FBD967
:101C5000F9DCF781B7308508D8FBD9F9DCF781B713
:101C6000B19CE493A3C39A6004DDC381B7DBDBB10D
:101C70008E6002812E7B08E493FAA3B16FDBF87AC1
:101C800030B16F752200752300B18EEAFCEBFDC305
:101C9000ED94FE400EB18E8A278B28ED30E0048A49
:101CA000828B83B18E7AC270D8C3ED94FE601950D6
:101CB000CEBD002BEC600F7520007521FF7529004B
:101CC000752A000200008100A827A9280809D80465
:101CD000D90281DCB192EA89AAF281CE0D81A3C337
:101CE000ED94035053EDA2E092007AC5C3E58294CF
:101CF00000E583941C508A200010438F02438F011B
:101D00008529B7852AB7F0300029A827A92808090E
:101D1000438F01538FFDD804D902A133C3E58394C7
:101D20001C4003A3A11689AAE28529B7852AB7F02A
:101D3000A3A116538FFC817F7AC1BD030CE493A34A
:101D4000FAB153DCF8B14B817F8181AA22AB23B178
:101D50006FEBFAEA6222752608C3E52313F523E543
:101D60002213F52250066323A0632201D526EAB18F
:101D7000DCB1DC75260AEAF4200102D285300102CA
:101D8000C285B1DCC3134002C201D526EB22B19259
:101D9000EAFB208502A192308502A197752608AE44
:101DA00024AF25C3EF13FFEE13FEB1E0B1DCC3EAAD
:101DB000133085024480FA30E703632201C3E52330
:101DC00013F523E52213F52250066323A0632201B5
:101DD000D526D9E52265236523F52222AE24AF2539
:101DE0000E0FDEFEDFFCD20122424C48656C6934E6
:071DF000373164F3300601F6
:00000001FF
